:030000000219FDE5
:03000B000200AA46
:03002B000201636C
:03005B000203009D
:030073000202ED99
:1000800002030406080C10182030406080040608A3
:100090000C10182030406080A0C00003070F1F0D17
:1000A0000D04050D050305030302C2AFC0D0C0E077
:1000B000206214E5256009E473E525F4F58AD2622F
:1000C000D0E0D0D0D2AF3285268AC262E526F46075
:1000D0003630682C20720DD0E0D0D0C283C294C2DA
:1000E00095D2AF32C283C294C295206F132066109E
:1000F000740CD5E0FDE57BB50704429021004280F9
:10010000D0E0D0D0D2AF32758A00C28DD262210049
:1001100001B9306805206602D28301B93068052034
:100120006602D29401B9306805206602D29501B901
:10013000C28030680A2066077408D5E0FDD28301CA
:10014000B9C28230680A2066077408D5E0FDD294EF
:1001500001B9C29730680A2066077408D5E0FDD25D
:100160009501B9C2AFC2AD53E6EFC0D0C0E0D2D363
:10017000D2AFC2CEE52A6007207449152A21C4787F
:1001800000790020742EE580307E01F430E502789D
:10019000FF53DACF207E0343DA20307E0343DA10A8
:1001A000C2D8C271E580307E01F430E50279FFC328
:1001B000E89970CB306103752A18207403752A18EA
:1001C000885CD27020740DE52B6004152B21D4437C
:1001D000DA01C2D82070024143A85C206102C270DB
:1001E0002074367982B70431C3E894F0400374F088
:1001F000F8E8C4540F28F87984B703024119C313EF
:10020000C3138721200802C313200A06C3C898F825
:10021000411928F8500374FFF88822E52D54066030
:1002200022206B1FE536C333C333F8E564C313C321
:1002300013F9C3952240028922E82522F5225003B2
:100240007522FF7882B60459852224A824C3E524A8
:1002500095614002A861C3E895634002A8638825C0
:10026000E56670024194C3E8AA669A5003E8FAE48E
:10027000F9EAC333FBE568F45B29400D2567F8E52F
:100280006760021567400B41940AC3E5679A500204
:10029000056778FF8826C26FC3E52694F84002D22E
:1002A0006FC3E52594404002D26420CF0AD0E0D04D
:1002B000D043E610D2AD32C2CF053A7801E52A60CC
:1002C00005307402152AC3E55C94014005755F0092
:1002D00041E3756000756900E55F2401F55F500337
:1002E000755FFFD0E0D0D043E610D2AD32C2AF533D
:1002F000E67F7592FA7593FFC260759104D2AF32B2
:10030000C2AF53E6EFC2ADC0D0C0E0C0F0D2D3D28E
:10031000AFA8FBA9FCC2D8307102616753DACF20C5
:100320007E0343DA10307E0343DA20D271E5803059
:100330007E01F420E502613E88278928A19453DAE2
:10034000CF207E0343DA20307E0343DA10C2D8C2C6
:1003500071307402A1807800E580307E01F430E5D0
:1003600002A180885CA16853DACF207E0343DA20A3
:10037000307E0343DA10C271206102814053DACF2C
:10038000207E0343DA10307E0343DA20C2D8D271D4
:1003900088578958C3E89555F8E99556F97B007E4A
:1003A000087A00C3E8948CE994005005755B0081DD
:1003B00032882178A2E6A8216055C3E894C8E99460
:1003C000005008E4D2E4FB7A0A810DC3E89468E99E
:1003D00094015008E4D2E3FB7A0F810DC3E894D076
:1003E000E994025008E4D2E2FB7A1E810DC3E8943E
:1003F000A0E994055008E4D2E1FB7A3C810DC3E802
:100400009498E994085008E4D2E0FB7A787E00C31F
:10041000E89559FCE9955AFD30E70AECF42401FC13
:10042000EDF43400FD755B00C3EC9AED9E5003754E
:100430005B018859895A8557558558567802A168B5
:10044000C3E89527F8E99528F9307C02A14C307B68
:1004500002A14C307A02A1452075028163E9FDE8D2
:10046000FC8182E9C313F9E813F8307902A145E968
:0F047000C313F9E813F8307802A145E9C313FD6F
:10047F00E813FC20612CC3EC941CED940240028124
:10048F0099ED701EC3EC94C850180529E529700228
:10049F001529C3E529940A5002A180755C00D2701A
:1004AF00A180E529600215297888E6F97400207F7C
:1004BF00087896B90302789EE624FAFEE43400FF2A
:1004CF00C3EC9EFCED9FFD9208B90310A2085007E4
:1004DF00207609D27681EB307602C276A2085016CA
:1004EF00B9030DECF42401FCEDF43400FD02050515
:1004FF0078007900A14CB90315EC33FCED33FDC343
:10050F00EC940AFCED9400FD50047C007D00C3ECDC
:10051F0094FFED9400400678FF7900A14CEC8572B2
:10052F00F0A4C5F0A2F733F879004003020568780C
:10053F00FF7900020568E9C313F9E813F8307C0E60
:10054F00E9600278FFC3E81338F8E43400F9C3E830
:10055F0094FFE99400400278FF885CD2702061021A
:10056F00A180741FF4552F4BF52FC274EB7002D27C
:10057F0074752A18307403752A0A306102A1942009
:10058F00740353DAFE207403752B06D0F0D0E0D03D
:10059F00D0D2AD43E6103279010205C479030205CA
:1005AF00C4790A0205C4791E0205C479640205C420
:1005BF0079C80205C47817E4D5E0FDD8FAD9F62238
:1005CF007A147B780205EB7A107B8C0205EB7A0D9F
:1005DF007BB40205EB7A0B7BC80205EB7902E4C210
:1005EF0082D5E0FDD294D5E0FDC294D5E0FDD28254
:1005FF00D5E0FDE920E002D28330E002D295E57329
:10060F00D5E0FDE920E002C28330E002C295749686
:10061F00D5E0FDD9C9EAF8D5E0FDD8FBDBBEC28233
:10062F0022C37C007D0075F00005F0EA33FAEB334E
:10063F00FB50F6EB13FBEA13FAC3E9FFE8FEE89A67
:10064F00F8E99BF95004EFF9EEF8B3EC33FCED3316
:10065F00FDD5F0DFEDF9ECF822E889F08A20D2D44D
:10066F00F8A9F07B0030F70B7BFFF42401F8E9F4D5
:10067F003400F9E88520F0A4ADF0F8E98520F0A466
:10068F00AFF0FEED2EF974003FFA7C04C3EA13FAC3
:10069F00E913F9E813F8DCF48BF030F70AE8F424E7
:1006AF0001F8E9F43400F9E889F0C2D4F8A9F0228E
:1006BF007882B6040302071AC3E55C940140030273
:1006CF0006E4852224E4F544F545F546F547F5485B
:1006DF00C26E02071A7882E6FCD26EE522F5237805
:1006EF003879C7AA40AB41C3EB13FBEA13FAEC14FA
:1006FF006013C3EB13FBEA13FAEC14146007C3EB9C
:10070F0013FBEA13FAD1308844894522C3E5449597
:10071F0023F8E5459400F9500CC3E89480E994FF61
:10072F00401602074BC3E8947FE994005003020779
:10073F004B787F790002074B788079FF8849894A87
:10074F0022E5492546F8E54A3547F9854A20E43040
:10075F000701F43548FA30E709C3EA94F04015026F
:10076F000789C3EA940F500302078978FF79FF7A4C
:10077F000F020789780079007AF0C3E5249561505C
:10078F000AC374019524500B0207A7E54A20E70E10
:10079F000207A7E54A30E706884689478A48227844
:1007AF00A5E6FAC3E54933F8E54A33F9D168E930EC
:1007BF00E70BC3E89480E994FF4013E1E1C3E894A9
:1007CF007FE994005002E1E1787F7900E1E17880E0
:1007DF0079FFE820E715C3E52398F84009C3E894AB
:1007EF000140030208087801020808E8F4240125F3
:1007FF0023F8400302080878FF884B2278A6E6FA10
:10080F00A847A948120668E930E70CC3E89401E944
:10081F0094FF401602083DC3E894FFE9940050038B
:10082F0002083D78FF790002083D780179FFE92041
:10083F00E715C3E54B98F84009C3E894014003025C
:10084F0008647801020864E8F42401254BF840039A
:10085F0002086478FF88242278FFC26420693D2053
:0E086F006A12D264C3E541940A4009C3E5252C
:10087D0094405002C26479A1E76023E541601F7482
:10088D00FF8541F0848539F0306A0375F005A4F8D1
:10089D00C5F0600278FFC3E895645002A8648863D0
:1008AD0022C3E5409440E5419401E56350031401F2
:1008BD00BF046002F563220208C72275E890227812
:1008CD0083E6FFE5E820ECF7A8BDA9BE0570C3E5FA
:1008DD007094084052757000E9FA79A0E76044EA17
:1008ED007007E571601B020902C3E895716010E5A0
:1008FD00715006600C1402090E0460F902090EE530
:10090D0071F571C3946D401B7561C0C394044013A0
:10091D00756180C39404400B756140C3940440031A
:10092D0075610075BB0922E5612410500274FFF555
:10093D00617982B70402215BC3A861E52498500256
:10094D00A824C3E895634002A86388258826E5702E
:10095D00B4070375BB1022743279A787F0A4C5F0D4
:10096D00A2F733F8C3E895614002A8618822882474
:10097D00882588268864227540007541F022C2AF13
:10098D0075C820A8CCA9CDAA3A30CF010A75C824C4
:10099D00D2AFAB3BAC3C883B893CC3E89BF8E99CB0
:1009AD00206908F9306702419721F4AD3D8A3DF980
:1009BD00EA9DFA600478FF79FFAE3EAF3F8B3E8C27
:1009CD003FA83BA93CC3E89EF8E99FF9C3E5411355
:1009DD00FBE54013FAE82AF540E93BF54150067571
:1009ED0040FF7541FF413EAA40AB41AC40AD417E59
:1009FD00047F02C3EB940440021E1FC3EB94084016
:100A0D00021E1FC3ED13FDEC13FCDEF7C3EA9CFAC7
:100A1D00EB9DFBEF6009C3E913F9E813F8DFF7EA83
:100A2D0028FAEB39FB8A408B4150067BFF8B408BBC
:100A3D0041C3EB94025002D2673069047F034169D0
:100A4D007892E6FFC3E537948240110FC3E53794E2
:100A5D00A040010FC3EF940640027F057E02E541E1
:100A6D00C4540FF9E541C454F0F8E540C4540F28BF
:100A7D00F8C3E89EFAE99400FB4009C3EA9402EB3F
:100A8D00940050047A02E4FB41E3AA40AB41EBC46D
:100A9D00FEEAC4540F4EFCC3EA9CFAEB9400FBC370
:100AAD00E813C313F8EA28FAEB3400FB8A408B41B4
:100ABD00C3EB94024002C2677802EBC4FE7B00EAEE
:100ACD00C4540F4EFAC3EA98FA4005C3940250027B
:100ADD007A027892E6FF30600241E38551928552A9
:100AED0093D26043E680C3E49AF8E49BF930670241
:100AFD00616FE8FAE9FBD3E913FDE813FC8851892E
:100B0D0052C3EF94036038EF20E00DE82CF8E93D77
:100B1D00F9ECFAEDFB020B38E828F8E939F9C3E8EE
:100B2D002402F8E93400F97AFE7BFFC3EF94034009
:100B3D000E8A538B54884D894E8C4F8D5061A388EE
:100B4D005389548A4D8B4E8C4F8D5030691275538D
:100B5D00F07554FF754FF07550FF7551F07552FFDC
:100B6D0061A3E8FAD3E813FC8851C3EF9403602026
:100B7D00EF20E007E82CF8ECFA618FE8282402F862
:100B8D007AFEC3EF940340088A53884D8C4F61A3BE
:100B9D0088538A4D8C4FE568C3335002646BF568FA
:100BAD0030600261AD753402D26043E680E52D54AC
:100BBD00066034A840A941C3E913F9E813F8C3E965
:100BCD0013F9E813F8306904E92440F9C2AF53E68C
:100BDD007F759100C3E498F594E499F595759104AA
:100BED00D26043E680D2AF22D265754300752000F6
:100BFD00306C03752040020C14D2657543007520CE
:100C0D0040306C0375200078017901206720E52DB7
:100C1D0054066002C2657914E541C313700104F8EE
:100C2D00C3941440027814306904781B791B20603A
:100C3D0010E543600C306903D53404D26D81B77172
:100C4D00B50543E59BF45440B5200281A1306909F7
:100C5D0008C3E899400118813B20650A08C3E8994B
:0D0C6D0040028114813BC265C2AF53E67F97
:100C7A007591003067127594007595FE759104D2CE
:100C8A006043E680D2AF8114AE40AF41C3E49EF523
:100C9A0094E49FF5958186C3E5339401500281144B
:100CAA003065028114D80281B5813BC26DC2AF534F
:100CBA00E67F759100855394855495759104854D09
:100CCA0092854E93D26043E680D2AFE52D540660FA
:100CDA0008206A020533020CF3306D0D206C0A20DD
:100CEA0065071581158102157B227800306405306D
:100CFA0065027801E53775F007A4F9E5F028F5F003
:100D0A00E9A2F013A2F113A2F213F537C3947850B3
:100D1A0003753778C3E53795384008D266C283C26F
:100D2A0094C295306002A12D854F92855093D2606E
:100D3A0043E68022207D16C2AF754202C282D2806B
:100D4A00306202D295D2AF759F43020F2DC2AF75A2
:100D5A004202C282D297306202D283D2AF759F43D7
:100D6A00020F2D307243207D20C2AF7542039001DD
:100D7A0041757B04C295C297306204D294A18BD28A
:100D8A0082D2AF759F53020F2DC2AF7542039001F5
:100D9A0041757B04C283C280306204D294A1ABD273
:100DAA0082D2AF759F33020F2D207D17C2AF7542D5
:100DBA000390011CC295306202D294D2AF759F5340
:100DCA00020F2DC2AF75420390011CC2833062022A
:100DDA00D294D2AF759F33020F2D207D16C2AF7504
:100DEA004204C280D297306202D294D2AF759F3346
:100DFA00020F2DC2AF754204C297D280306202D26E
:100E0A0094D2AF759F53020F2D307243207D20C2BA
:100E1A00AF754205900130757B01C294C28230627F
:100E2A0004D283C131D280D2AF759F43020F2DC243
:100E3A00AF754205900152757B80C294C2823062BE
:100E4A0004D295C151D297D2AF759F43020F2D207C
:100E5A007D17C2AF754205900112C294306202D268
:100E6A0083D2AF759F43020F2DC2AF754205900121
:100E7A0026C2943062EBD295D2AF759F43020F2DF2
:100E8A00207D16C2AF754206C297D282306202D264
:100E9A0083D2AF759F53020F2DC2AF754206C2802F
:100EAA00D282306202D295D2AF759F33020F2D30B3
:100EBA007243207D20C2AF754201900152757B803A
:100ECA00C283C280306204D295C1D7D297D2AF759D
:100EDA009F33020F2DC2AF754201900130757B011D
:100EEA00C295C297306204D283C1F7D280D2AF755D
:100EFA009F53020F2D207D17C2AF75420190012624
:100F0A00C283306202D295D2AF759F33020F2DC2CF
:100F1A00AF754201900112C295306202D283D2AFFC
:100F2A00759F53C26622900110757B00C283C294DA
:100F3A00C295C280C282C297C262227880760908AC
:100F4A0076090876040876FF0876030876FF08769D
:100F5A0009087603087601087601788C7601087606
:100F6A00FF0876FF0876FF0876FF0876FF08760303
:100F7A000876FF0876FF0876FF0876250876D008F7
:100F8A0076280876500876040876FF0876020876EE
:100F9A000008767A0876FF08760108760108760056
:100FAA00087603087600227887E6FFC272BF03023A
:100FBA00D2727888E6C394036008C27DE630E10203
:100FCA00D27DC27E7889E630E102D27EC3EF9402F6
:100FDA006008758E01D273020FE9758E00C2732202
:100FEA007880E6149000809378A5F67881E61490CC
:100FFA0000809378A6F67886E61490008D9378A7F9
:10100A00F67886E6F539C394025003753902789C5E
:10101A00E67538FFB402037538A0B4030375388245
:10102A0078A3E61490009A93F566120F302222787C
:10103A0096E6FA7897E6FB7888E6B40305C3EB945C
:10104A000EFB307F047A007BFFC3EB9AFCC39482C9
:10105A0050027C827572000572EC8572F0A4C3E5B9
:0F106A00F0947D40F222D27F11391205B57A0041
:101079007B007C101205ABE55C2AFA74003BFBDCB3
:10108900F37C04C3EB13FBEA13FADCF7FEC27F110E
:101099003922E5EF20E6037520000520903FFFE5A2
:1010A90020146006901DFF1460009304600375EF1F
:1010B9001253D9BF7581C043FF801205A675EF028F
:1010C90043B203E5B3240220E70DF521E5E320E06F
:1010D900068521B343E301120F307580F275A40D23
:1010E90075F13F75D4DF75904F75A5B075F2F07540
:1010F900D50075A60175E241120F30E4F8F6D8FD66
:10110900756801120F451215CC78988673753001F0
:10111900C2AF1205BF1205CF1205B51205D61205C9
:10112900B51205DD1205B5C2AF78FA79FA3085072F
:10113900D9FBD8F7021C00120FB1120FEA113811AE
:101149003978988673120F3075881075890275C8B9
:101159002475910475D84075A82275B80275E69072
:10116900759B80759D0075D10E75BC5875BB097549
:10117900BA1175E8801205A6D2AF1208C4753600F7
:1011890053DACF207E0343DA20307E0343DA10435B
:10119900DA01C2D8C2711205BFD2617B037A0CE5AC
:1011A9005B70077A0CDB030211301205B52070035E
:1011B900021130C270E55CC3940240E1E52F541F6F
:1011C900855E5DF55EB55DD5DAD5C26153DACF20AE
:1011D9007E0343DA20307E0343DA10C2D8C2717825
:1011E900A2E67008D274E52F54E0F52FC27575296F
:1011F900001205BA307409C3E529940A4002D27570
:101209001205AB78023074027800C3E55C9840F0AF
:10121900C2AF1205CF1205CF1205CFD2AF1205BF4B
:10122900754C007888E6B4030261081205AB788C26
:10123900E6C394015003021308E530C39401500337
:10124900021308207435C3E55C94FF5003021308A8
:10125900C2AF1205E4D2AF1205BAC3E55C940150DE
:10126900EFC2AF1205CF1205B01205CFD2AF1205EA
:10127900BAC3E55C94FF40E90217747F02D27F117B
:10128900391205BAC2AFC27F1139AE5CC3E55C94AD
:101299007FD2AF40741205A6C2AF1205E4D2AFDF08
:1012A900DC1170C3EE7897F61205BF12160E1216EE
:1012B900F77F0AD27F11391205BAC2AFC27F11393D
:1012C900AE5CC3E55C947FD2AF50E61205A6C2AF0F
:1012D9001205CF1205B01205CFD2AFDFD61170EECD
:1012E90024037896F61205BF12160E121726120558
:1012F900BA1139C3E55C94FF5002414C021774C31B
:10130900E55C954C4003855C4C1205BA78017988F7
:10131900E7B403027805C3E55C984002412CC2AFEB
:101329001205E41205E41205E4D2AF1205BF7530C7
:1013390000E4F531F5320531E531F4703F053278D5
:101349009AE67819146012783214600D787D146069
:101359000878FA146003753200C3E53298401D120B
:101369000F301205A6153275310078998673C2AF10
:101379001205E4D2AF789886731205BA1205B0E562
:101389002A7005307402213078012074027806C36E
:10139900E55C9840A17888E6C3940360031205BA16
:1013A900E52A7003021130C2AF120F30E4F522F5BD
:1013B90023F524F525F526F567D2AF7885E6C333FD
:1013C900F565E4F544F545F546F547F548F570F555
:1013D9002CF52DF53775700875BB101205A6120886
:1013E900C8E5E820ECFBA8BDA9BEE97001F8887141
:1013F9001208CC75700875BB10120FB1C2AF7561B8
:10140900FF120964852261852262852263D2AF7544
:101419002201752401752501752601856069756AA2
:10142900017888E6B40307C27D307602D27DD2689E
:10143900D269753300120E8A120EB9120984120983
:101449008B12098412098B120984120C061206BF29
:10145900120CF4120D3E12098B120BF5306E0312A9
:0E146900071B2067031208673067031208AEE6
:10147700120CF4120D6D12098B120C06306E03124A
:101487000750120CF4120DE412098B120BF5306E93
:10149700031207AE120CF4120E1312098B120C066C
:1014A700306E0312080B120CF4120E8A12098B12FB
:1014B70008C8120BF5120CF4120EB91208CC120957
:1014C7008B306932856461856462856069756A01FC
:1014D70079187A0CC3E53399400FC269D26A8A3505
:1014E7008564618564630214FDC3E55C9401400370
:1014F700021453021583306A1D206C1AE5351470E7
:1015070006C26AD26B8153F535C3E55C940140038B
:1015170002145302158375360078FA79A4E760023E
:101527007803C3E55F985054307404E52A604D781A
:1015370088E6B40317207D05207607A1533076028D
:10154700A153206C07D26C856461819278F0306C6E
:10155700058564617820C3E5419850028153306C5A
:101567001BC26CC27D307602D27DD26A7535128578
:10157700646181530536E55C6002A186753600C259
:10158700AF120F307887E6FE7602120FB17887EE3A
:10159700F6E4F522F523F524F525F526F565752CF2
:1015A70000752D00D2AF1205BA120F3078A4E6608D
:1015B70006D283D294D295307409C3E53694044099
:1015C700022130613A901A0D7820121650E520B4A6
:1015D700550CA3121650E520B4AA030215EE120FFC
:1015E7004512160E02160D901A0378807B0A121602
:1015F70050A308DBF9901A0F788C7B19121650A3A9
:1016070008DBF9901A2822C2AF12168F12166990BA
:101617001A00740E121655A37406121655A37415E4
:10162700121655901A0378807B0A121654A308DB0A
:10163700F9901A0F788C7B19121654A308DBF9124C
:1016470016A2121680901A2822E493F622E6438FF8
:1016570001538FFD75EF0275B7A575B7F1F0538F7D
:10166700FE22438F02438F0175EF0275B7A575B749
:10167700F1901A0DF0538FFC22901A0D7455D15525
:10168700901A0E74AAD155227A3079D07820901A00
:1016970040D150E520F709A3DAF7227A3079D090C4
:1016A7001A40E7D15509A3DAF922AB74A875BB0133
:1016B700027980BB02027981BB03027982BB0402F3
:1016C7007984BB05027986BB06027992BB0702794A
:1016D70087BB080279A3BB0902799CBB0A027988F8
:1016E700BB0B027989E8F7227C051205BFDCFB22D8
:1016F700C2AF1205CF1205D61205DD1205E4120599
:10170700B01205CF1205D61205DD1205E41205B099
:101717001205CF1205D61205DD1205E4D2AF22C29B
:10172700AF1205E41205DD1205D61205CF1205B07A
:101737001205E41205DD1205D61205CF1205B01207
:1017470005E41205DD1205D61205CFD2AF22AE741D
:10175700AF75C2AF1205CF1205CF1205CF1205B074
:10176700DEF21205E41205B0DFF8D2AF22D1F7D1CD
:10177700EFD1EF757401757501757600F1557C052C
:10178700AD5C1205BFC3ED955C70F5C3E55C9401D4
:10179700400AC3E55C94FF40320217B0D1B1D10EC5
:1017A700D1F7C2AF75EF12D1EFDCD50576C3E57679
:1017B7009403500280C6D1EF0575E5741490009F1D
:1017C70093F808C3E57598500280AED1EFD1EF05C5
:1017D70074C3E574940C5002809C120F45D10EC25D
:0617E700AF75EF12D1EF17
:0319FD0002109B3A
:101A00000E0615090904FF03FF0903010155AA0188
:101A1000FFFFFFFFFF03FFFFFF25D0285004FF0259
:091A2000007AFF0101000300FF40
:101A400023416C69676E424C333558232020202097
:101A500023424C48454C4923463333302320202031
:101A60002020202020202020202020202020202076
:101C0000C2AFC2D353D9BF7581C043B20343FF8073
:101C1000752438752503B1C975EF0275E24043F1AB
:101C20002053A4DF75D4FFD2857DFA780379E67C52
:101C300010752200752300901DD67B0675249875BB
:101C400025013085028142208508D8FBD9F9DCF7CF
:101C500081B4308508D8FBD9F9DCF781B4B189E4C7
:101C600093A3C39A6004DDC381B4DBDBB17B600264
:101C7000812B7B08E493FAA3B15CDBF87A30B15C8A
:101C8000752200752300B17BEAFCEBFDC3ED94FEE9
:101C9000400EB17B8A278B28ED30E0048A828B834B
:101CA000B17B7AC270D8C3ED94FE601350CEBD00F4
:101CB00025EC60097520007521FF0200008100A855
:101CC00027A9280809D804D90281D3B17FEA89AAB3
:101CD000F281C50D81A0C3ED94035049EDA2E092BD
:101CE000007AC5C3E5829400E583941C50902000DF
:101CF00010438F02438F0175B7A575B7F1F030001F
:101D00001FA827A9280809438F01538FFDD804D99C
:101D100002A12089AAE275B7A575B7F1F0A3A10DBC
:101D2000538FFC817C7AC1BD030CE493A3FAB140CC
:101D3000DCF8B138817C817EAA22AB23B15CEBFA5E
:101D4000EA6222752608C3E52313F523E52213F57D
:101D50002250066323A0632201D526EAB1C9B1C986
:101D600075260AEAF4200102D285300102C285B14B
:101D7000C9C3134002C201D526EB22B17FEAFB2082
:101D80008502A17F308502A184752608AE24AF2587
:101D9000C3EF13FFEE13FEB1CDB1C9C3EA13308513
:101DA000024480FA30E703632201C3E52313F523DD
:101DB000E52213F52250066323A0632201D526D91C
:101DC000E52265236523F52222AE24AF250E0FDE22
:101DD000FEDFFCD20122424C48656C693437316326
:041DE000F3300601D5
:00000001FF
